:100000008A0103282D29831686018312A301083053
:1000100083122302013003180301003C0319512805
:1000200086012308A000003C031D18280614482858
:1000300083122008013C031D1F28861448288312C0
:100040002008023C031D2628061548288312200894
:10005000033C031D2D288615482883122008043CE4
:10006000031D34280616482883122008053C031D6A
:100070003B288616482883122008063C031D422888
:100080000617482883122008073C031D48288617B6
:10009000FA308312A10002208A110A128312A30AE5
:1000A000072883128601A30108308312230201303E
:1000B00003180301003C03199D282308A000003CFD
:1000C000031D64280614942883122008013C031D94
:1000D0006B288614942883122008023C031D722882
:1000E0000615942883122008033C031D79288615E1
:1000F000942883122008043C031D802806169428A7
:1001000083122008053C031D872886169428831235
:100110002008063C031D8E28061794288312200809
:10012000073C031D94288617FA308312A100022091
:100130008A110A128312A30A542883128601FA3004
:10014000A10002208A110A123F3083128600FA3081
:10015000A10002208A110A12063083128600FA30AA
:10016000A10002208A110A125B3083128600FA3045
:10017000A10002208A110A124F3083128600FA3041
:10018000A10002208A110A12663083128600FA301A
:10019000A10002208A110A126D3083128600FA3003
:1001A000A10002208A110A127D3083128600FA30E3
:1001B000A10002208A110A12073083128600FA3049
:1001C000A10002208A110A127F3083128600FA30C1
:1001D000A10002208A110A126F3083128600FA30C1
:1001E000A10002208A110A126F3083128600FA30B1
:1001F000A10002208A110A12773083128600FA3099
:10020000A10002208A110A127C3083128600FA3083
:10021000A10002208A110A12393083128600FA30B6
:10022000A10002208A110A125E3083128600FA3081
:10023000A10002208A110A12793083128600FA3056
:10024000A10002208A110A12713083128600FA304E
:10025000A10002208A110A1205288E308312A20002
:10026000000000000000000000000000A20B322986
:0A0270000000A10B2D29000008007A
:00000001FF
